:020000040000FA
:1000000064008B138B120B11532882000000000038
:10001000080042348434A434833401342434C33497
:10002000043402347434A3344434C2348234E334A8
:100030006434D43443340334813423341434633487
:100040009434B434C434FD347D343D341D340D3423
:1000500005348534C534E534F5347B3418347B34C9
:100060000C347B3406347B340334603403344C3436
:1000700003343C3403342834033420344D344834BE
:100080007A342034003455345334423400344C3400
:1000900053344234003450345234473400344334FF
:1000A00041344C3400347621013005148510051597
:1000B0000512F920061A9628FD309800FF309900A5
:1000C000BF309A0000309B007F21A7214F300A22C9
:1000D0000D3013220A301322061B76289A0A031DBC
:1000E0007528990A031D7528980A8728861B872872
:1000F000FF309A07031C8028990A031D8028980A5C
:10010000FF309907031C8528980AFF309807061EC0
:1001100064284F21061E64281808940019089500C9
:100120001A0896001B0897001030F12105151030B1
:10013000C621140898001508990016089A00170897
:100140009B00F920B901BE11BE12061AC0284F212A
:10015000061AC0287F211008940011089500120883
:10016000960013089700A7214B300A220D30132266
:100170000A301322061EAA284F21061EAA28BE16E0
:10018000861FC528061FCE28D128061FC828CA28C2
:100190000030D228BE15B9090430D228BE15083067
:1001A000D2280C30BE1AD628C621D728F1217F21AB
:1001B000861EDB2820210521901FE0282021B90977
:1001C000A721BE1DE9283918E7284330E828473021
:1001D0000A220D3013220A30132205114921492128
:1001E00049214921492149214921492149214921BF
:1001F0009628060D0E392D3E0520C500060D0E3938
:100200002D3E013E0520C700080017089307031C78
:100210001029920A031D1029910A031D1029900A22
:1002200016089207031C1829910A031D1829900A21
:1002300015089107031C1D29900A1408900708004F
:100240009009910992099309930A031D2E29920A94
:10025000031D2E29910A031D2E29900A0800302122
:10026000900C910C920C930C9013080018088C00C1
:1002700019088D001A088E008E0F3C299C218D0FC5
:100280003C298C0F3C29003442308C008C0B4629D1
:1002900000340A308D0044218D0B4B2900340301BA
:1002A0008E0049218E0B512900342030BA00B40150
:1002B000B501B601B701B801343084000530BB0088
:1002C000333080078019F039801B0F398002840A8F
:1002D000BB0B6029930D920D910D900DB80DB70DCC
:1002E000B60DB50DB40DBA0B5C2908008316373076
:1002F000810008308500FF30860083120800051257
:100300000B11810190019101920193010516362193
:100310000512000000000000000000009C21010800
:100320009200831601120000011683129303010844
:1003300012060319912908000B1DA4290B11910A1B
:10034000031DA329900A080000000000A3292F2103
:10035000552135080F39031DB02920301322B1294A
:10036000C321360EC3212E3013223608C321370E87
:10037000C3213708C321851DC129380EC321380880
:10038000C3213D300A2A0F39303E132A83128900D7
:100390000C3A0319DA29D5219400D4219500D421EF
:1003A0009600D42197000800890A83160814831246
:1003B000080808000430C6211408900015089100B0
:1003C00016089200170893000830C6210521302135
:1003D0001008940011089500120896001308970061
:1003E0000800831289001408FD211508FC21160855
:1003F000FC211708FC210800890A880083160815CB
:1004000055308900AA30890088148818052A0812F6
:1004100083120800890009080520FF3903190828FC
:100420001322890A0B2AC800C522861D0800480825
:10043000853E03182A2A1A3E0318522A063E03183C
:100440002A2A1A3E0318522A073E03182A2A0A3E6D
:100450000318542A4808203A031D2E2A48082C3A2B
:10046000031D362ACC30C9000630582A48082E3AD7
:10047000031D3E2A5430C9000630582A4808043A61
:10048000031D462A5030C9000530582A4808203A32
:10049000031D512A47088F00732273228F0B4C2AA9
:1004A00073220800093E552A233E0520C90007395A
:1004B000CA005B2A7322C90D031C602A6A226A22C1
:1004C0006A22CA03031D5A2A47088F0073228F0B22
:1004D000662A08004508C60085147C2285107C2207
:1004E000C60B6C2A08004508C60000007C220000EC
:1004F0007C22C60B752A0800CE308C008C0B7E2A1D
:100500000034C100030EC2000408C3005730C522E6
:100510003D30C5224108BB222030C5222030C522F3
:100520005330C5225230C5223D30C5224208BB227D
:10053000B72284010008BB222030C522840A0408A7
:100540000F39031DA52AB722AA2A0339031DAA2A97
:100550002030C5220408B03E031D9A2AB722B722D4
:1005600043088400420E8300C10E410E08000D3086
:10057000C5220A30C52AC400440EBF2244080F39E0
:10058000F63E031CC42A073E3A3EBF000830C000B6
:100590000510E730013E031DCA2ABF0C0318D22AFA
:1005A0000510D32A0514C00BC92AE730013E031DEC
:0E05B000D62A0514CD30013E031DDB2A0800BB
:02400E00F23F7F
:1042000000000000000000000000000000000000AE
:10421000000000000000000000000000000000009E
:08422000FD00FF00BF000000DB
:00000001FF
